S018000064656D6F70726F675F786D63343730302E737265633D
S3150C0040000088FE1F054200089D4200089D420008DC
S3150C0040109D4200089D4200089D42000800000000D9
S3150C0040200000000000000000000000009D42000897
S3150C0040309D420008000000009D420008CD4F00087C
S3150C0040409D4200089D4200089D4200089D420008C2
S3150C0040509D4200089D4200089D4200089D420008B2
S3150C0040609D42000800000000000000000000000057
S3150C0040709D420008000000009D4200089D42000879
S3150C0040809D4200089D4200089D4200089D42000882
S3150C0040909D4200089D4200089D4200089D42000872
S3150C0040A09D4200089D4200089D4200089D42000862
S3150C0040B09D4200089D4200089D4200089D42000852
S3150C0040C09D4200089D4200089D4200089D42000842
S3150C0040D09D4200089D4200089D4200089D42000832
S3150C0040E09D4200089D4200089D4200089D42000822
S3150C0040F09D4200089D4200089D4200089D42000812
S3150C0041009D4200089D4200089D4200089D42000801
S3150C0041109D4200089D4200089D4200089D420008F1
S3150C0041209D4200089D4200089D4200089D420008E1
S3150C0041309D4200089D4200089D4200089D420008D1
S3150C0041409D4200089D4200089D4200089D420008C1
S3150C0041509D4200089D4200089D4200089D420008B1
S3150C004160000000000000000000000000000000003D
S3150C0041709D4200089D4200089D4200089D42000891
S3150C0041809D4200089D4200089D4200089D42000881
S3150C0041909D4200089D4200089D4200089D42000871
S3150C0041A09D4200089D4200089D4200089D42000861
S3150C0041B09D4200089D4200089D4200089D42000851
S3150C0041C09D4200089D4200089D4200089D42000841
S3150C0041D09D4200089D4200089D4200080000000018
S3150C0041E09D4200089D4200089D4200089D42000821
S3150C0041F09D420008000000009D42000800000000DF
S3150C004200EE11AA55DFF874D01D4880471D4C1E4D83
S3150C004210AC4209DA21686268A368043BA2BFC8589D
S3150C004220D050FAE70C34F3E7184B194CA34208DAD2
S3150C00423019685A680020043AA4BF8850FBE7083373
S3150C004240F4E7144880471448804700002850000CB7
S3150C0042500088FE1F000000002850000C0088FE1F7E
S3150C004260000000000088FE1F8000000000000020F7
S3150C0042700000000000000020000000000088FE1F67
S3150C0042802D4500084C4200086442000864420008B0
S3150C0042907C420008DD4F00085D4F0008FEE7000079
S3150C0042A082B00023019303E000BF019B013301930D
S3150C0042B0019B8342F8D302B0704700BF72B60D4B18
S3150C0042C00D4A9A60BFF34F8F62B6D3F8882042F43A
S3150C0042D07002C3F888205A6922F008025A6107490D
S3150C0042E041F214028B5823F00F0343F004038B5056
S3150C0042F0704700BF00ED00E00040000800100058B9
S3150C00430000487047001BB70010B51E4BDB6813F452
S3150C004310803F27D01C4BDB6813F0010F02D1FFF74F
S3150C004320EFFF00E01948184B1B6813F0040F11D06F
S3150C00433015498A68C2F303628B68C3F306238C683B
S3150C004340C4F30644611C02FB0112B0FBF2F203FB40
S3150C004350022208E00C4B9B6803F07F030133B0FB91
S3150C004360F3F200E0094A0749C868C0B20130B2FB53
S3150C004370F0F3086900F001000130B3FBF0F0044BD8
S3150C004380186010BD004600501047005000366E01F4
S3150C004390C0FF032070B5574B1B6813F0010F09D1F2
S3150C0043A0544A536843F001035360524B1B6813F095
S3150C0043B0010FFAD0504B1B6813F4007F08D04E4AFD
S3150C0043C0936843F40073936041F64C50FFF768FF13
S3150C0043D04A4C636843F40023636040F6C410FFF74D
S3150C0043E05FFF636823F4803323F002036360444B5E
S3150C0043F05B6813F0300F21D0103C636823F47023F4
S3150C00440023F030036360FFF77BFF3E4BA3FB0023D7
S3150C0044101B0D013B626842EA03436360374BDA6863
S3150C00442022F00102DA605A6822F400325A60334BE9
S3150C0044301B6803F46073B3F5607FF8D12F4B5A6891
S3150C00444042F001025A605A6842F010025A602E4A33
S3150C0044509A605A6842F040025A605A6822F010027A
S3150C0044605A605A6842F480225A60244B1B6813F037
S3150C004470040FFAD0214A536823F0010353601F4BF3
S3150C0044801B6813F0010FFAD1204C4FF00113E360B7
S3150C004490002666612661266266620323E3611C4B75
S3150C0044A0A3611C4BA362154D6B6823F040036B6034
S3150C0044B0194BAB604FF41660FFF7F2FE174BAB606F
S3150C0044C04FF46160FFF7ECFE154BAB604FF4965062
S3150C0044D0FFF7E6FE134BAB6041F27070FFF7E0FEA0
S3150C0044E0114BAB604FF4E150FFF7DAFE6660FFF755
S3150C0044F00BFF70BD004200500044005010470050A6
S3150C004500004700506BCA5F6B002F0B010046005032
S3150C0045100500010003002001002F0501002F0301F7
S3150C004520002F0201002F0101002F000110B54FF0E2
S3150C0045300053044C0FCB84E80F00FFF7BFFEFFF7C8
S3150C00454029FF10BDC4FF0320F0B48B081F1D50F8C3
S3150C004550276001F00305ED00F824AC4026EA0404BC
S3150C00456040F82740466F4F000324BC4026EA04045B
S3150C0045704467184CA04203D004F58074A04207D1BE
S3150C004580046E012606FA01F124EA0101016617E020
S3150C00459054688C404460CC08103450F8247001F0F8
S3150C0045A00701890007268E4027EA060640F8246094
S3150C0045B050F82470167A06FA01F1394340F82410A3
S3150C0045C0043350F823101278AA400A4340F82320EB
S3150C0045D0F0BC7047008E0248030F20F0704003EBCE
S3150C0045E043039B00014A9850704700BF1444005087
S3150C0045F0034B1868034B5B6903F00103D840704703
S3150C004600C0FF032000460050030F20F0704003EB60
S3150C00461043039B00014A9850704700BF4846005020
S3150C0046202DE9F04142F2107E0027BC46012638E007
S3150C0046300B6803EB83035B00B3FBF6F34D68B3FB2C
S3150C004640F5F4374AA2FB0482D20802EB820252002E
S3150C004650A21A052A05D9324AA2FB0442D208013213
S3150C00466003E02F4AA2FB0442D2082AB102EB8204D1
S3150C0046706400B3FBF4F304E0294AA2FB0323DB0832
S3150C0046800122AB4201D35B1B00E0EB1A142A07D8BC
S3150C0046909E4505D9B3F57A7F06D39E461746B44692
S3150C0046A00136402EC4D901E01746B44642F2107EBC
S3150C0046B00126402212E042F2107302FB0333B3FBD5
S3150C0046C0F7F30C899C4201D81D1B00E0E51AAE4598
S3150C0046D001D9AE461646A34202D3013A022AEAD8BB
S3150C0046E0BB1B026842F040020260023B1B0303F450
S3150C0046F0E0434A89013A9201D2B21343721E120266
S3150C00470002F4706213430CF1FF3C0CF03F0C43EACD
S3150C0047100C030361036823F040030360BDE8F081DA
S3150C004720CDCCCCCCD0F8C43113F4407FFAD10131C6
S3150C004730120442F0020242EA0161C0F8C411704749
S3150C00474038B50446074D2846FFF75EFF2846FFF7A7
S3150C00475043FF236823F001032360236813F0020F41
S3150C004760FBD138BD10000010D0F8C83123F00F0370
S3150C0047701943C0F8C8117047D0F8C80100F00F00F3
S3150C004780704700BF08B5FFF7F7FF012802D00228D3
S3150C00479003D005E0FFF72CFF08BDFFF7B1FD08BD00
S3150C0047A0002008BDF8B504460E461546FFF7C8FFAF
S3150C0047B020463146FFF7D8FF2046FFF7E3FFB0FB54
S3150C0047C0F5F2C2F58062002A38BF002240F2FF37AC
S3150C0047D0BA4228BF3A46C2F58061B0FBF1F1AE0988
S3150C0047E08009B602B6FBF0F3BB4228BF3B4603FB7F
S3150C0047F000F0800A691AA5EB801081428CBF00205C
S3150C004800012000B1134608B1012100E00221E26843
S3150C00481022F4434222F0FF02E260E26843EA81336B
S3150C0048201343E360F8BD00BF037E012B17D1036869
S3150C0048302022DA6101680B6823F07062037B1B0689
S3150C00484003F0706313430B60036802691A61036813
S3150C00485042695A610368034ADA61002070470320F3
S3150C004860704700BF40002800026802F13843A3F5E8
S3150C004870A833990AC3F344131B0243EA41339168E4
S3150C00488021F47F419160026891680B439360037E2B
S3150C004890012B2FD810B503682022DA61C37913F0E7
S3150C0048A0200F0ED1426802F0604343EA824302684D
S3150C0048B09361826802F0604343EA82430268D360E4
S3150C0048C005E0036842689A6103688268DA60044608
S3150C0048D0037E012B06D1FFF7A7FF23684FF000627A
S3150C0048E0DA6103E003684FF40062DA612368024A76
S3150C0048F0DA6110BD704700BF4000A0060368D96995
S3150C004900DA69C2F3800211F4006F0FD182B91A6909
S3150C00491002615A694261D969DA69C2F3C00211F0BF
S3150C004920040F07D0002AF2D10020704703207047ED
S3150C004930022070470020704730B48B08043350F8BF
S3150C004940235001F00301C900F8248C4025EA040425
S3150C00495040F8234050F823408A40224340F8232055
S3150C00496030BC704770B505460E4600F0E3F8F47996
S3150C00497004B9102428463168224600F035F8B3797C
S3150C004980013B64080134240244EA430343F44033F4
S3150C00499043F00103EB633379013B1B0643F481734C
S3150C0049A06B6373792BB16A6B013B42EA03436B630E
S3150C0049B005E06A6B3379013B42EA03436B634FF4C0
S3150C0049C0A063AB634FF0FF33EB6433892B6470BD8C
S3150C0049D0D0F80C3113F0E06F02D1406D80B2704705
S3150C0049E0D0F81C0180B2704763293BD9002A3BD012
S3150C0049F02DE9F04115460C460646FFF7F9FD1B4915
S3150C004A00A1FB00377F09A1FB0431480940F2FF3EA8
S3150C004A104FF0010CE046714611E001FB07F305FB74
S3150C004A2000F2B3FBF2F39C0AC3F30903B4F5806FEF
S3150C004A3004D2734502D29E46A44688460139002903
S3150C004A40EBD148F4004333617269094B1340013DC5
S3150C004A5043EA85230CF1FF3C43EA0C4373610020C7
S3150C004A60BDE8F08101207047012070471F85EB518E
S3150C004A70EF8000FC30B4D0F8084124F0E064C0F8B4
S3150C004A800841D0F80851064C2C4041EA032343EA6E
S3150C004A90026244EA0203C0F8083130BC704700BF1A
S3150C004AA0C0C0FFF830B4D0F80C4124F0E064C0F874
S3150C004AB00C41D0F80C51074C2C4041EA032343EA35
S3150C004AC0026244EA020343F08053C0F80C3130BC56
S3150C004AD0704700BFC0C0FFEF10B5114B984208D10C
S3150C004AE04FF40060FFF790FD4FF40060FFF774FD84
S3150C004AF010BD0C4B984207D10B4C2046FFF784FD9A
S3150C004B002046FFF769FD10BD084B984206D1084CAC
S3150C004B102046FFF779FD2046FFF75EFD10BD00BF6E
S3150C004B2008000340080002488000001008400248B4
S3150C004B300001001010B50446154B984203D003F53E
S3150C004B400073984203D11348FFF7C6FF14E0124BCB
S3150C004B50984203D003F50073984203D10F48FFF730
S3150C004B60BBFF09E00E4B984203D003F50073984245
S3150C004B7002D10C48FFF7B0FF0323E360E36813F0A0
S3150C004B80010FFBD0236C23F00F03236410BD00BF71
S3150C004B9000000340080003400000024808000248D9
S3150C004BA00040024808400248704700BF2DE9F04318
S3150C004BB08BB04FF46143019308238DF808308DF8C0
S3150C004BC0093001258DF80A5010278DF80B70002638
S3150C004BD0ADF80C601C4C204601A9FFF7C3FE8DF8FE
S3150C004BE01C6008954FF002098DF82490DFF85C8064
S3150C004BF04046042107AAFFF7A7FC90238DF8103036
S3150C004C0005958DF81890404605210DEB0702FFF728
S3150C004C109BFCE36923F007032B43E36120463946EB
S3150C004C2004222B46FFF726FF2046314604222B464C
S3150C004C30FFF738FF236C23F00F0343EA09032364C1
S3150C004C400BB0BDE8F08300BF0000034000810248B2
S3150C004C5030B58BB0FFF7CCFC044600E06400434B48
S3150C004C609C42FBD900E06408414B9C42FBD841486E
S3150C004C7001212246FFF796FD01943F4B02934FF418
S3150C004C80FA53ADF80C300123ADF80E303B4C2046F0
S3150C004C9001A9FFF7C5FC236843F040032360236892
S3150C004CA043F001032360364B36481860DA7902214B
S3150C004CB061F38712DA71596840F2676464F31C0178
S3150C004CC059609A6864F31C029A60090E6FF34511D9
S3150C004CD0D971120E42F02002DA72C26842F000520A
S3150C004CE0C26008221A73002305E0254A1A440021E3
S3150C004CF011740133DBB2072BF7D921480025057651
S3150C004D00FFF7B2FD1B4801210A46FFF70BFD1B4CB2
S3150C004D10236823F040032360236823F001032360F8
S3150C004D200AAA02F80C5D184D28460D21FFF70CFC5B
S3150C004D3090238DF810300123059302238DF818303B
S3150C004D4028460C2104AAFFF7FFFB236843F0400317
S3150C004D502360E36823F0070343F00203E360236850
S3150C004D6023F0400323600BB030BD00BFFF1AB70021
S3150C004D70000E27070040014820A107000043014808
S3150C004D805088FE1F2050014800810248074BD3F87B
S3150C004D90143113F0080F07D110B504460348FFF77A
S3150C004DA017FE2070012010BD002070470000034044
S3150C004DB008B5FFF7FBFEFFF74BFF08BDBFF34F8FA0
S3150C004DC00549CA6802F4E062044B1343CB60BFF397
S3150C004DD04F8F00BFFDE700BF00ED00E00400FA05B1
S3150C004DE008B51F4B1B789BB91E48FFF7CFFF012850
S3150C004DF035D11C4B1B78002B31D000F0E1F81A4B47
S3150C004E0018600122164B1A700022184B1A7008BD36
S3150C004E10164B1B7816481844FFF7B8FF012814D117
S3150C004E20124A13780133DBB213700E4A127893428E
S3150C004E3015D100220A4B1A700A4B5B78FF2B0ED148
S3150C004E40084B9B785BB9FFF7B9FF00F0B9F8064B36
S3150C004E501B686433984202D90022014B1A7008BDB4
S3150C004E607088FE1F0488FE1F0088FE1F4888FE1FE0
S3150C004E700588FE1F00B583B0174B1B68DB6913F062
S3150C004E80010F1BD01448FFF739FD60B1002210E06A
S3150C004E90114A1A44117C02AA1A4402F8081C01335E
S3150C004EA0DBB2012201E0002213460B49097B994231
S3150C004EB0EED8094B1B680121D96100E0002242B1F2
S3150C004EC09DF80030FF2B04D19DF801300BB9FFF78C
S3150C004ED075FF03B05DF804FB5088FE1F08B5FFF79D
S3150C004EE07FFFFFF7C7FF08BD10B5054C204608210C
S3150C004EF08022FFF721FD4FF08073636010BD00BF69
S3150C004F000085024808B500F05BF80D4B1B68C31A08
S3150C004F10B3F5FA7F13D30B4B1B783BB90122094B24
S3150C004F201A704FF48072084B5A6006E00022054B4B
S3150C004F301A704FF08072044B5A60014B186008BD12
S3150C004F407488FE1F7888FE1F0085024808B5FFF797
S3150C004F50DBF9FFF7C9FF00F011F808BD08B5FFF73C
S3150C004F60F5FFFFF725FFFFF7CDFFFFF7B7FFFAE7D2
S3150C004F70014B1860704700BF7C88FE1F08B50C4BB0
S3150C004F801B680C4AA2FB03239B09013BB3F1807FF0
S3150C004F9009D2094A5360FC21084B83F823100023DD
S3150C004FA09360072313600020FFF7E2FF08BD00BFE4
S3150C004FB0C0FF0320D34D621010E000E000ED00E0CE
S3150C004FC0014B1868704700BF7C88FE1F024A1368A5
S3150C004FD001331360704700BF7C88FE1F70B50E4B03
S3150C004FE00E4CE41AA41000251E46A54204D056F811
S3150C004FF0253098470135F8E7FFF7D6FD084C094BE5
S3150C005000E41AA41000251E46A54204D056F82530F5
S3150C00501098470135F8E770BD0088FE1F0088FE1F13
S30D0C0050200088FE1F0088FE1F2C
S70508004205AB
